S31508001800A0090020D9180008E7180008E9180008F8
S3150800181000000000000000000000000000000000BA
S315080018200000000000000000000000000119000888
S31508001830000000000000000003190008C93600086F
S3150800184011410008071900080719000807190008B8
S3150800185007190008071900080719000807190008DA
S31508001860071900087528000807190008071900084D
S3150800187007190008071900080719000807190008BA
S3150800188007190008000000000000000007190008FA
S3150800189000000000071900080719000807190008C2
S315080018A0000000000719000807190008753B000822
S315080018B007190008071900080719000800000000A2
S315080018C0EE11AA550348854600F0B0FC00480047CB
S315080018D0FD520008A00900200B4880F308880B4831
S315080018E080470B480047FEE704207146084202D0AD
S315080018F0EFF3098001E0EFF30880714603F076FB09
S31508001900FEE7FEE7FEE7FEE7A0090020C537000868
S31508001910C518000830B50B460146002020220124D0
S3150800192009E00D46D5409D4205D31D469540491B05
S315080019302546954040191546521E002DF1DC30BD4E
S3150800194070B500242546002801DA01244042002902
S3150800195001DA01254942FFF7DDFFAC4200D04042DB
S31508001960002C00D0494270BD03460B439B0703D0A9
S3150800197009E008C9121F08C0042AFAD203E00B7846
S315080019800370401C491C521EF9D27047D2B201E0BE
S315080019900270401C491EFBD270470022F6E710B5BC
S315080019A013460A4604461946FFF7F0FF204610BDBF
S315080019B0F8B502464A40D40F42004B0052085B086D
S315080019C09A4202D20246084611464A0023D0C30D5F
S315080019D04A00DDB2120EAD1A202D35DA490201266B
S315080019E0490AF6058A19002C00D0524220214F1BBD
S315080019F01146B9402A411018C20D9A4221D0002C2E
S31508001A0017D0012D08DCDA05801AD20F8019D20703
S31508001A10DBB200F021FBF8BDDA05801A012340008D
S31508001A201B06C01880185A428018CA0F104349006E
S31508001A3007E04908C2071143DA05801A80194008E9
S31508001A40801800F001FBF8BD61000122511A001B45
S31508001A50F7E70122D2075140AAE70122D2075040F0
S31508001A60A6E7024670B54A40D30FDB0740002DD0E3
S31508001A704A002AD0010E140E000212020919400A61
S31508001A80520A8418E50104465443000A120A2E0431
S31508001A905043A4194219200CC543AA18120C012553
S31508001AA0AD03521C521912047F39240400D0521C6B
S31508001AB0104301D44000491EC2B20C06C0092018C2
S31508001AC0401C4008802A02D003E0002070BD400870
S31508001AD04000002900DA0020184370BD70B50246A0
S31508001AE04A40D50F40004A00ED0740085208002832
S31508001AF014D0002A12D0C40DD30D41020120C0050E
S31508001B005202490A520AE41A091812187D349142F7
S31508001B1001D3641C00E04900002C01DA002070BDE6
S31508001B200023914201D3891A03434008490000283B
S31508001B30F7D100290AD0914202D10121C90705E04F
S31508001B40914201D2012101E00121C943E005C018F3
S31508001B50401900F079FA70BDF0B5074608465840B6
S31508001B6087B0C00F049048000E465900400849083F
S31508001B70BC1A884105D2384631461E4617460B46DA
S31508001B8002465800400810434CD0300D03904005DB
S31508001B905900400D490D0590401A0290402872DA06
S31508001BA018030121000B09050843019004980092C7
S31508001BB0002805D0019952420020884100920190E0
S31508001BC0029840210A1A0199009800F009FA054678
S31508001BD00C466B4607CB00F024FAC0197141039AEC
S31508001BE00E0D0023D71756401A467A40164344D09E
S31508001BF0049A002A2DD0029A012A039A15DC1205A6
S31508001C00C01A914101263605001C7141D20F059E66
S31508001C10D2070093019202962A46234600F062FAFA
S31508001C2007B0F0BD38463146FAE71605224A0F4690
S31508001C30B218C01AB74101210905001C4F41001806
S31508001C407F41114618187941E20F10436D19644116
S31508001C5013E0E2076D0815436408C2071443039AA4
S31508001C6001261205C01A91413605001C7141CE079E
S31508001C70400830434908C01851412A46234600F017
S31508001C8024FACDE7FFE7049801224000C117121A8B
S31508001C9000238B4104983146C417381AA141EEE750
S31508001CA030B40124E407634030BC55E730B401245E
S31508001CB0E407614030BC4FE70000E0FFF0B51FB411
S31508001CC088B00B990998002448400999C00F490023
S31508001CD049080991C0070B990090490049080B91DA
S31508001CE009990898A64608431CD00B990A980843F0
S31508001CF018D0099801244000420D4800410D099862
S31508001D0024050003000B204309900B980003000BE1
S31508001D1020430B9050181C49401800220190144685
S31508001D20104605E0002001460DB0F0BD032801DA93
S31508001D30034600E003239C46C11A0AAE0AE05F0088
S31508001D4008ADED5B4F00F75B7D430027AA187C4181
S31508001D50491C5B1E6145F2DD410004AB5A52210461
S31508001D60120C0A43240C401C0828DFDB0198029059
S31508001D700099704601910090059B049A0799069868
S31508001D8000F0B0F9D0E700000DFCFFFFF0B50C46F7
S31508001D905C4085B0E40FE40703944C000026640811
S31508001DA059009446490802460296224321D06246C3
S31508001DB00A431ED06200570D4A000E032303550D31
S31508001DC0012402462C492405781B1B0B360B4018A8
S31508001DD023432643614600901C46501AB44103D358
S31508001DE00098401C009002E0921800985B41002879
S31508001DF003DA0020014605B0F0BD002001210905DF
S31508001E000746864611E064461D46141BB54106D3AF
S31508001E106546521BB341744607430C43A646CD0795
S31508001E2040084908284392185B4105460D43EAD104
S31508001E301046184313D0604619465040714008436F
S31508001E4006D06046101AB34106D20122002306E0E6
S31508001E5000220123DB0702E00122D2435310009837
S31508001E6074460105381C6141029C039D00196941AD
S31508001E7000F02BF9BFE70000FD030000C217C10FF1
S31508001E80504010B54018CA079623002100F0E4F820
S31508001E9010BD10B500229623114600F0DDF810BDDE
S31508001EA00EB505490291002100910A460B4601919B
S31508001EB000F018F903B000BD3304000041004002E9
S31508001EC00122400AD205090E80187F2901DA00206E
S31508001ED07047962903DC9622511AC84070479639EE
S31508001EE0884070474A0009030123090B1B0519435B
S31508001EF0094B10B5520D9A4201DA002010BD064B67
S31508001F0034339A4203DC9A1A00F07AF810BD034972
S31508001F105118884010BD0000FF030000CDFBFFFFED
S31508001F20C20FD207400040080BD0C10D0723DB01C2
S31508001F30C91840020905400A1143C208400711435F
S31508001F407047002001467047CB0FDB07490010B5E4
S31508001F50490802460A4307D00A0D07240903E40183
S31508001F60090B121B002A01DC002010BDC900440F12
S31508001F700C43C100E018D205801800F065F810BDC2
S31508001F80F0B51FB40646002082B0054640240191EC
S31508001F9000901BE0019922460F46304600F030F8C3
S31508001FA0049A059B801A994110D310461946224671
S31508001FB000F016F8361A8F410197224601200021B3
S31508001FC0009F00F00DF838184D4100902046641E19
S31508001FD00028DFDC019B00982946324607B0F0BD91
S31508001FE010B5202A04DB0146203A9140002010BD96
S31508001FF0914020239C1A0346E3401943904010BDA4
S3150800200010B5202A04DB0846203AD040002110BD2E
S315080020100B46D340D0402024A21A914008431946C3
S3150800202010BD10B5202A06DBCB170846203A10410A
S31508002030C1170B4306E00B461341D0402024A21AD1
S3150800204091400843194610BD002904DA401C49008E
S3150800205001D140084000704770B40024050C05D132
S315080020601024000402D1002921D01124050E01D123
S3150800207000020834050F01D10001241D850F01D186
S315080020808000A41C002801DB4000641C002908D03D
S3150800209020252E1B0D46F540A14000D001212943DD
S315080020A0084301061B1B000ADB1D02D5002070BC75
S315080020B07047DB05181880180029F8DA401C490013
S315080020C0F5D170BC40084000704710B5002B08DAFF
S315080020D00024401C614192185B411A4301D1400813
S315080020E0400010BDF0B51FB482B005460C0003D001
S315080020F0084602F04DF802E002F04AF8203002469F
S31508002100009021462846FFF76BFF049B059A044674
S315080021100F4618431143084314D0184610431BD0E2
S31508002120009840210A1A18460599FFF769FF0546DF
S315080021300E46009A05990498FFF752FF084305D002
S31508002140012004E02046394607B0F0BD0020C1173B
S3150800215005430E432C43374300990E986305401AEE
S315080021607905E40A00220C43FD0A0A3002D500204C
S315080021700146E9E70105101969410C9C0D9D0019F6
S315080021806941FFF7A2FFDFE7FEB500231A461B1ACF
S315080021908A4103DB0020014603B0F0BD4A000D0367
S315080021A001212D0B0905520D0D43D10702D1001847
S315080021B06D41521E5110FF31FF310131002704468F
S315080021C03E4638460097019102460121002009053E
S315080021D0FFF716FFC3197141F818324684468E4632
S315080021E04A4161462846611A904104D36046241A3A
S315080021F0954176461F46241900986D41401C00906B
S315080022003428E1DDF91930467041091BA84103D28B
S315080022100022D243134601E0002213460198010525
S31508002220381C7141FFF751FFB6E70000064C01253F
S31508002230064E05E0E36807CC2B430C3C9847103460
S31508002240B442F7D3FFF742FB0C6400082C6400087D
S3150800225010B50446002C08D101210920C00600F05B
S31508002260D5FD002000F0DAF84BE0012C05D102215B
S315080022700920C00600F0CAFD43E0022C05D104215E
S315080022800920C00600F0C2FD3BE0032C05D1082159
S315080022900920C00600F0BAFD33E0042C05D1102150
S315080022A00920C00600F0B2FD2BE0052C05D120213F
S315080022B00920C00600F0AAFD23E0062C05D140211E
S315080022C00920C00600F0A2FD1BE0072C05D18021DD
S315080022D00920C00600F09AFD13E0082C04D101215C
S315080022E00A4800F093FD0CE0092C04D102210748A6
S315080022F000F08CFD05E00B2C03D11021034800F0FB
S3150800230085FD204600F08AF810BD0000000400484C
S31508002310FEB50020009001900290002428E00025D8
S315080023200DE006206843274940186100405AA1007D
S315080023306A4651584018A1005050681C85B2142DA1
S31508002340EFDBA1006A4650581421FFF7E3FA28216B
S31508002350484361001C4A515A3C225143461864219D
S315080023603046FFF7D7FA6100174A5052601C84B20C
S31508002370032CD4DB15488079002822D012484088DF
S315080023801349884203DC10488088884208DD0F48D4
S315080023902038C07B002803D101210C482038C1739E
S315080023A0094840880A2803DB074880880A2808DA8B
S315080023B006482038C07B002803D10121034820386D
S315080023C0C173FEBD100400202C01002090030020DC
S315080023D0E60F000000B587B001A800F0AFF80121AC
S315080023E0480200F0E3FF00200190702002900120CF
S315080023F08002039000200690059001A9064800F087
S3150800240031F80121044800F021F80121024800F0C2
S3150800241011F807B000BD00000024014010B50446BD
S31508002420072300222146024800F038F810BD0000B4
S3150800243000240140002904D0426801231A4342605F
S3150800244003E042685208520042607047002904D0EF
S31508002450826808231A43826003E0826808239A4345
S315080024608260704742680B4B1A4042600B684A68A4
S315080024701A4343681A4342608268074B1A408260CF
S315080024800B694A691A438B681A4383681A43826040
S31508002490704700000FBCFFFF8FF1F9FFF0B5044647
S315080024A00D4616461F463F073F0F2B46082B0FD9EA
S315080024B01B071B0F083B606F9A000F21914088434A
S315080024C06067606F99003A468A40104360670BE080
S315080024D0206F9A000F21914088432067206F99004A
S315080024E03A468A4010432067E0680121A94088439C
S315080024F0E060E0680121A9400843E060012080030C
S315080025002840002803D0012000F020F807E0012029
S31508002510C0032840002802D0012000F017F8F0BDBB
S31508002520002905D08268FF2301331A43826004E03C
S315080025308268FF2301339A43826070470021016055
S31508002540416081600173016141617047002806D0CE
S31508002550064949680C221143044A516005E00349BB
S3150800256049680C229143014A516070470024014092
S3150800257010B523480078012835D100202049087075
S315080025802049088013E01F48008840001E49095A60
S315080025901E480088062250431D4A8018194A128888
S315080025A05200815217480088401C16490880154871
S315080025B000880328E7DB7E2001F0B6FD022000F044
S315080025C02BF901211348FFF7ABFF10480088401C80
S315080025D00E49088008460088142804DB0020088075
S315080025E001200D4908700C480078002806D0FFF72E
S315080025F08FFE00200849087000F052FC10BD00004C
S315080026003801002052010020DC030020540100207C
S31508002610100400200024014032010020FFB583B0D9
S315080026200C46029400200190002726E000261CE0B4
S31508002630721C039951430846791CFFF76BF9054646
S31508002640A54201D9281B00E0601B05460298A8424E
S3150800265004D902950598067006980770029800280E
S3150800266002D10120019002E0761C402EE0D300BF83
S315080026700198002800D002E07F1C042FD6D300BFA3
S31508002680029807B0F0BD000000BF00BF00BF00BF42
S3150800269000BFBFF34F8F00BF00BF00BF0648074902
S315080026A0C86000BF00BF00BFBFF34F8F00BF00BFA9
S315080026B000BF00BF00BFFDE70400FA0500ED00E01B
S315080026C010B500F001F810BD10B5234800780028B1
S315080026D017D1224800F0F2FE01283CD11F480078A5
S315080026E0002838DD1D480078402834DC01F015FA4A
S315080026F01B4908600120184908700020194908700C
S3150800270029E0164A17490978491C501800F0D6FEE0
S31508002710012816D113480078401C124908700F4842
S3150800272000780978884216D100200B4908700B48B2
S315080027304078FF280FD10B48007802280BD1FFF705
S31508002740A3FF01F0EAF9064909686431884202D90B
S3150800275000200149087010BD0501002098030020DB
S31508002760080100200401002010B586B004460121A6
S31508002770880300F01BFE0121480400F0F7FD012242
S315080027800921C80600F02DFB01220A210920C006EE
S3150800279000F027FB01A801F0C6FA0194302168462B
S315080027A0018100214181818101821821C18101A90C
S315080027B0184801F075FA0121164801F04EFA05A8E5
S315080027C000F065FB01214902684681820121817575
S315080027D01821C17505A90920C00600F0B5FA01211E
S315080027E08902684681824821C17505A90920C00663
S315080027F000F0AAFA1B2168460170032141700121E5
S31508002800817000F07FFD01220221024801F03DFAA5
S3150800281006B010BD0038014001B5044900980860AB
S3150800282000BF024800680028FBD108BD0C01002043
S31508002830014600220E4B1A61CA005A6100229A61AB
S3150800284005221A6100BF0A4A1069C207D20F002A78
S3150800285004D0012212040240002AF4D0044A126964
S3150800286052085200024B1A6100229A617047000012
S3150800287000E000E010B500210448FFF751FE0220F1
S3150800288000F04AF801200249087010BD00240140F2
S315080028903801002000B589B00121084600F066FD20
S315080028A01A4800F045F801A800F08EF8184801907B
S315080028B01848029000216846017303200490684670
S315080028C00175802141754900C18289000183202153
S315080028D08176090281830021C183018401A90B48FD
S315080028E000F04CF80121094800F01CF801220221E9
S315080028F0064800F039F8092168460170022141703E
S315080029000121817000F0FEFC09B000BD08000240FC
S3150800291000240140DC03002001494860704700009C
S31508002920000002400268520852000A4302607047DB
S3150800293010B504462068400840002060002020604A
S315080029406060A060E060E1B2084608380521FEF73D
S31508002950E1FF01460F2088400249496808430149BA
S31508002960486010BD00000240002A03D003680B43EC
S31508002970036002E003688B430360704710B50A7A68
S315080029808B7D1A430B7C1A434B7C1A434B8A1A439A
S315080029908B8A1A430B8B1A434B8B1A430368094CD1
S315080029A023401A43026002680123DB039A438B8B98
S315080029B01A430260CA6842600A6882604A68C2604E
S315080029C010BD00000F80FFFF002101604160017209
S315080029D0C16001744174418281828175018341839A
S315080029E08183704770B506460C4621460A4800F0B2
S315080029F04BF90546002D01D1401E70BD064885429B
S31508002A0002D10648051B00E02D1B22462946304602
S31508002A10FEF7AAFF2046F0E700F4000800FC0008CD
S31508002A2070B506460C4621460A4800F02DF90546BB
S31508002A30002D01D1401E70BD0648854202D10648C8
S31508002A40051B00E02D1B224629463046FEF78CFF63
S31508002A502046F0E7008000080088000870B50646A2
S31508002A600C4621460A4800F00FF90546002D01D10B
S31508002A70401E70BD0648854202D10648051B00E087
S31508002A802D1B224629463046FEF76EFF2046F0E704
S31508002A90009000080098000870B505460C462246C6
S31508002AA00249284600F0B1F8204670BD00F4000837
S31508002AB070B505460C4622460249284600F0A5F898
S31508002AC0204670BD0080000810B504460848006915
S31508002AD00221084306490861084644610069402105
S31508002AE0084303490861034800F00EF910BD0000C9
S31508002AF000200240FF0F00000C48C068C007C00F46
S31508002B00002801D0012070470848C0680421084001
S31508002B10002801D00220F6E70448C06810210840C2
S31508002B20002801D00320EEE70420ECE7002002404D
S31508002B30034800698021084301490861704700007D
S31508002B400020024030B504460D46054800690121BB
S31508002B5008430349086125800F2000F0D5F830BDE9
S31508002B600020024010B57E2001F0DEFA064800F08B
S31508002B700FF87E2001F0D8FA044800F009F87E2004
S31508002B8001F0D2FA10BD000000F400080080000829
S31508002B9010B5044600F0ACF82046FFF795FFFFF79E
S31508002BA0C7FF10BD70B503460125002208E0500096
S31508002BB01C5A0748844201D0002506E0501C82B200
S31508002BC0CE0F761876109642F1DC00BF284670BD07
S31508002BD0FFFF0000F8B505460E46144600F088F8D3
S31508002BE07E2001F0A1FA002707E029883046FFF782
S31508002BF0A9FFB61CAD1C781C87B2E10F091949104C
S31508002C00B942F2DCFFF794FFF8BDF8B507460C4663
S31508002C1015462946204600F037F80646002E0DD1FF
S31508002C202046FFF7B5FF012080022018FFF7B0FF06
S31508002C302A4621463846FFF7CDFF24E001208002C8
S31508002C402018401BB0420AD1012080022018FFF745
S31508002C509FFF2A4631463846FFF7BCFF13E001209E
S31508002C60C0022018401BB04208D12046FFF790FF4B
S31508002C702A4631463846FFF7ADFF04E02A46314674
S31508002C803846FFF7A7FFF8BDF8B505460E462F46A6
S31508002C90E807C00F002801D000BFFEE73146012033
S31508002CA0C002FEF74DFE002901D000BFFEE7002452
S31508002CB00BE020467043471931463846FFF772FF46
S31508002CC0012800D108E0601C84B231460120C00208
S31508002CD0FEF736FEA042ECDC00BF31460120C002FA
S31508002CE0FEF72EFEA04200D100273846F8BD0000A8
S31508002CF0024803494860034848607047230167450E
S31508002D0000200240AB89EFCD10B5024600BFFFF7A1
S31508002D10F3FE0346521EFF2400E0641E002CFCD17D
S31508002D20012B01D1002AF2D1064800697721884390
S31508002D30044908613420C860002A01D1052010BD65
S31508002D401846FCE700200240F8B50246CD782F0762
S31508002D503F0FCD7810263540002D01D08D782F43B2
S31508002D601446002011E085062B0E0D8801268640A4
S31508002D703540002D07D025680F269E40B5433E46B0
S31508002D809E4035432560451CE8B20828EBDB141D38
S31508002D900D882D120095002011E085062B0E0125C1
S31508002DA08540009E3540002D07D025680F269E4099
S31508002DB0B5433E469E4035432560451CE8B2082883
S31508002DC0EBDBCD78282D04D155690E88354355613E
S31508002DD006E0CD78482D03D115690E88354315616F
S31508002DE0F8BD70B54D07EB0E082902DA0546203501
S31508002DF001E0054624352C460F269E402568B54336
S31508002E0016469E403543256070BD000038B5044619
S31508002E100D460920C006844203D10121480400F06A
S31508002E20A5FA1148844203D10121000200F09EFA56
S31508002E300E48844203D10121000200F097FA0C489B
S31508002E40844203D10121080500F090FA684600F093
S31508002E501EF868460580012181700021C170694607
S31508002E602046FFF771FF38BD0004004800080048F7
S31508002E70000C0048024690680840002801D001204E
S31508002E8070470020FCE741617047016170470021E7
S31508002E90C9430180022181700421C1707047000076
S31508002EA0F0B58FB00025002600200D900C907E20EE
S31508002EB001F03AF900241AE06100954A505AFEF7E3
S31508002EC0E8FF94490790FEF709FE0746FFF728F83A
S31508002ED00022914B09910890FEF7F0FE0B910A909B
S31508002EE0FFF732F8A1008D4A5050601C84B2032CBB
S31508002EF0E2DB8A498868FFF713F8894A894B059106
S31508002F000490FEF7CDFE0022874B07910690FEF748
S31508002F103DFF864A864B09910890FEF7C7FE0B913E
S31508002F200A90FFF711F805467C494868FEF7F8FF4E
S31508002F307B4A7C4B05910490FEF7B2FE00227A4B41
S31508002F4007910690FEF722FF784A794B0991089077
S31508002F50FEF7ACFE0B910A90FEF7F6FF06462846EA
S31508002F60FEF7DEFF00226C4B05910490FEF79EFEED
S31508002F700991089029466F48FEF773FD0746FEF744
S31508002F80CFFF07910690099B089AFEF7FFFE0B9163
S31508002F900A90FEF7D9FF684908603046FEF7C0FF79
S31508002FA000225D4B05910490FEF780FE099108907A
S31508002FB031466048FEF755FD0746FEF7B1FF079113
S31508002FC00690099B089AFEF7E1FE0B910A90FEF718
S31508002FD0BBFF5A4908605A49088BFEF761FF594AF0
S31508002FE0594B03910290FEF769FE0022574B059153
S31508002FF00490FEF7CBFE099108905149088BFEF71D
S3150800300048FF0746FEF78CFF0022504B01910090BF
S31508003010FEF7BCFE0591049047480068FEF780FF5E
S3150800302003910290059B049AFEF73AFE07910690D3
S31508003030099B089AFEF7AAFE0B910A90FEF784FFF1
S315080030400D903F49488BFEF72BFF3E4A3E4B0391B6
S315080030500290FEF733FE00223C4B05910490FEF7E2
S3150800306095FE099108903649488BFEF712FF0746E8
S31508003070FEF756FF0022354B01910090FEF786FEBB
S31508003080059104902D480068FEF74AFF03910290C7
S31508003090059B049AFEF704FE07910690099B089A79
S315080030A0FEF774FE0B910A90FEF74EFF0C90284827
S315080030B00D99FEF77DFC0746FEF700FF25490860D7
S315080030C023480C99FEF774FC0746FEF7F7FE2249DB
S315080030D00860224800881F4909684018C003010C87
S315080030E01E48018040881C4909684018C003010C25
S315080030F01A484180094908681949FEF7B2FC07468B
S31508003100FEF7DCFE81B21548C1800FB0F0BD0000A5
S315080031102C01002000F07F45000008400404002030
S31508003120333333333333C33F0000284025068195B4
S31508003130438BD43F0000484340010020440100204F
S31508003140F0010020091B9E5E29CB703F00408F408E
S315080031500000C841480100204C01002070030020EF
S315080031600000C842014800687047000010010020AE
S315080031700348006803490978401801490860704700
S31508003180100100201801002008B50121480400F0AC
S31508003190EDF80121880400F0E9F86846FFF777FEA4
S315080031A00121C903684601804821C1706946092082
S315080031B0C006FFF7C9FD6846FFF769FE0121090346
S315080031C0684601804821C17069460920C006FFF794
S315080031D0BBFD6846FFF75BFE402168460180042177
S315080031E0C17069460148FFF7AFFD08BD00040048F5
S315080031F010B50121C9030920C006FFF73BFE0028C8
S3150800320008D12148007D002808D101211E480175F2
S31508003210417303E000211C48417301751B4880680F
S315080032207D21090188422CD900201849886000218F
S31508003230154841732030807900281CD1082114488C
S31508003240FFF723FE10488038408803280BDA0E481B
S315080032504088822804DA01210B482030817102E077
S3150800326001210948C1730848007B012809D10020BB
S315080032700649486005E000200449486000210248E4
S3150800328001730148407B10BD70030020B001002087
S315080032900004004808B50121480400F067F8012138
S315080032A0880400F063F86846FFF7F1FD29216846AF
S315080032B00180012181701021C17069461048FFF70D
S315080032C043FD962168460180012181701021C17055
S315080032D069460920C006FFF737FD10210920C006F8
S315080032E0FFF7D1FD80210920C006FFF7CCFD01219B
S315080032F00348FFF7C8FD08210148FFF7C6FD08BDCA
S31508003300000400488178002925D0174903221202B3
S315080033108918027892109200895802789207D30E7B
S31508003320FF229A40914342789207120E03789B0730
S31508003330DB0E9A4011430C4A03231B02D21803786A
S315080033409B109B00D1500178CA06D20E01219140EC
S31508003350054A116007E00178CA06D20E012191409C
S31508003360014A80321160704700E100E0002905D06B
S31508003370054A52690243044B5A6104E0024A5269FB
S315080033808243014B5A61704700100240002905D05C
S31508003390054AD2690243044BDA6104E0024AD2695B
S315080033A08243014BDA61704700100240002905D0BC
S315080033B0054A92690243044B9A6104E0024A9269FB
S315080033C08243014B9A6170470010024010B500F025
S315080033D031F804494968F02211400909024A515C4A
S315080033E0C84010BD00100240DE00002010B5FFF7EF
S315080033F0EDFF05494968072212021140090A034AE6
S31508003400515CC84010BD000000100240DE000020DC
S3150800341010B5FFF7DBFF054949680722D2021140BC
S31508003420C90A034A515CC84010BD0000001002409A
S31508003430DE000020F8B51E4840680C210840042824
S3150800344002D008282ED101E01A4C2DE01848403049
S315080034500069C007C00F00280AD015484030006927
S3150800346002210840002801D0134802E0114800E074
S31508003470104807460E4840300069FF2109040840F5
S31508003480000C451C0A48403000690721090208401B
S31508003490000A461C3946694308463146FEF73AFA99
S315080034A0044601E0034C00BF00BF2046F8BD0000FB
S315080034B00010024000127A0000093D0070B504466B
S315080034C000250221074800F0CEFB002808D0054851
S315080034D000F022FC20700221024800F0BCFB012506
S315080034E0284670BD0038014010B500F001F810BD3F
S315080034F000B585B062480068012108436049086044
S3150800350000BF5F480068022108400028F9D05D48DE
S315080035105D4908605D480068102108435B490860FA
S3150800352008460068C008C000086057490968481E70
S315080035305749FEF7EFF9049054480068049949077B
S31508003540490F0843514908604D48406851490840A9
S315080035504B494860084640689021084348494860F6
S31508003560084640684860484800684649884207D97E
S3150800357043484068052109020843414948600BE071
S31508003580414800684449884206D93D4840680121B7
S31508003590890208433A4948606B4601AA3A480168D5
S315080035A03E48FFF73BF836484030006980088000FF
S315080035B033494031086108460069400840000861FF
S315080035C0684600784007400F029068460079400632
S315080035D0400E03902A48C069890508432849C861EE
S315080035E02748403000692E4908402549403108617E
S315080035F003980004029909020843214940310969E0
S3150800360008431F49403108611D4800680121090621
S3150800361008431B49086000E000BF194800680121FB
S31508003620490608400028F7D01548406880088000F9
S315080036301349486008464068022108431049486013
S3150800364000E000BF0E4840680C2108400828F8D161
S315080036500120FFF7EDF80A48406810218843084919
S3150800366048600120FFF7E4F8054840688021884350
S31508003670034948600120FFF7DBF805B000BD0000EC
S315080036800010024000A24A04F00000200020024078
S3150800369000366E010FC0FFFF0051250200127A00A6
S315080036A0FFF800FF042806D10649096904221143D8
S315080036B0044A116105E00349096904229143014A54
S315080036C01161704700E000E010B5FFF751FD3A4878
S315080036D00088401C3849088008464068401C4860F5
S315080036E036480068002804D034480068401E33492C
S315080036F008603348407B012805D12F488068401C64
S315080037002D49886002E000202B4988602C48807A81
S31508003710012805D128480069401C2749086102E0AC
S315080037200020254908612648007C012805D1224841
S31508003730806B401C2049886302E000201E4988638C
S315080037401D4948680A21FEF7E5F8002923D11C48D7
S315080037502030C1788078814208DD19482030807889
S31508003760401CC1B216482030817014E0144820303D
S31508003770C1788078814200D10DE011482030C178A7
S315080037808078814207DA0E4820308078401EC1B220
S315080037900B48203081700A4820308079022804D0EE
S315080037A0074820308079032804D10348006B401C61
S315080037B00149086310BD0000B00100200C0100207B
S315080037C07003002010B51648006801210843144903
S315080037D00860084640681349084011494860084689
S315080037E00068114908400E4908600846006801212A
S315080037F0890488430A49086008464068C3210904C1
S31508003800884307494860084600680849084004494B
S3150800381008609F2000048860FFF766FE10BD000060
S31508003820001002400CC0FFF8FFFFF6FEFFFF8F00F6
S3150800383008B501214804FFF799FD02220121092054
S31508003840C006FFF7CEFA0221684601801821C1702A
S315080038500121817069460920C006FFF775FA012122
S315080038604804FFF783FD022211460920C006FFF728
S31508003870B8FA0421684601801821C17001218170B7
S3150800388069460920C006FFF75FFA08BD30B587B05C
S3150800389004460D4601210846FFF778FD04A800F006
S315080038A033F905946846058200210183817681747F
S315080038B004A90120800700F0F1F8684600F0D2F864
S315080038C060216846017001214170002001900021A5
S315080038D06846017269460120800700F057F8694674
S315080038E00120800700F08AF80821C80600F07EF853
S315080038F00821C80600F0B0F84021080600F038F89C
S315080039004021080600F03CF80121880700F00AF873
S315080039100121880700F01EF80121880700F00EF83B
S3150800392007B030BD002904D0026880231A4302601C
S3150800393003E0026880239A4302607047002904D096
S31508003940026801231A43026003E002685208520023
S3150800395002607047002905D0426C0123DB031A4335
S31508003960426404E0426C0123DB039A4342647047D5
S31508003970826907231B039A430B021A438261704725
S31508003980C26970239A430A43C261704710B58269B7
S3150800399007231B039A430B781B021A4382610A7A90
S315080039A012014B781B011A43036A3024A3431A43B6
S315080039B002624A6882630C4A904213D14A7A12011B
S315080039C08B781B011A43036AC024A3431A43026275
S315080039D04A8992008B899B001A4343682401A343B2
S315080039E01A43426010BD0000002C01408269012381
S315080039F0DB029A430B021A438261704710B5C2690B
S31508003A0070239A430B781A43C2610A7A12024B78DA
S31508003A101B021A43036A03242402A3431A430262BD
S31508003A204A68C2630B4A904213D14A7A12028B78CB
S31508003A301B021A43036AA400A3431A4302624A8973
S31508003A4012018B891B011A434368A400A3431A4336
S31508003A50426010BD002C0140C26908239A430A43FC
S31508003A60C261704700210170417081704160017226
S31508003A70417241818181704701229207904201D1AA
S31508003A80816301E08AB282637047012292079042FD
S31508003A9001D1C16301E08AB2C26370470268032399
S31508003AA01B029A430B891A430260134A904206D0B6
S31508003AB001229207904202D0104A904205D102682C
S31508003AC070239A438B781A4302600B4A904205D0BA
S31508003AD00B4A904202D00B4A904205D1026B120A59
S31508003AE012028B7A1A4302634A68C2620A888262A1
S31508003AF00122426170470000002C0140000400408A
S31508003B0000440140004801400021C94341600021AA
S31508003B100180018181708172704710B5FFF722FB21
S31508003B2010BD000070B5FFF751FC05467D21C900A0
S31508003B30FDF7F0FE0446601E0C49884200D90CE0E9
S31508003B40601E0B4948610321081F00F047FB00204F
S31508003B50074988610720086100BF0420FFF7A2FD16
S31508003B600021481E00F03AFB70BD0000FFFFFF0071
S31508003B7000E000E010B50221154800F07DF80028A5
S31508003B8024D0134800F0C8F8C4B21248807A002836
S31508003B9003D1204601F0E2F814E00E48807A0228A4
S31508003BA010D10C48C07A00280CD10B488079AA2875
S31508003BB004D10948C47101210648C172AA2C01D151
S31508003BC0054884710221024800F045F810BD00003E
S31508003BD000380140700300209404002010B5044604
S31508003BE02146054800F09CF800BF0121024800F074
S31508003BF03AF80028F9D010BD0038014070B50546DE
S31508003C000E4600247E2000F08FFA00BF20E0042C28
S31508003C1019DD701EA04216DD285D7E2806D17D209E
S31508003C20FFF7DCFF5E20FFF7D9FF0FE0285D7D2850
S31508003C3005D1FFF7D3FF5D20FFF7D0FF06E0285D2B
S31508003C40FFF7CCFF02E0285DFFF7C8FF601C84B2CF
S31508003C50B442DCDB70BD416170478269520852008C
S31508003C600A4382617047024690680840002801D0DE
S31508003C70012070470020FCE70246D068084000286B
S31508003C8001D0012070470020FCE7002A03D0036911
S31508003C900B43036102E003698B430361704700002D
S31508003CA070B504460D460026E06930218843297917
S31508003CB00843E061E06944218843A9790843E06143
S31508003CC0E06980088000297A0843E061A069182124
S31508003CD0884369890843A061A06904218843297B30
S31508003CE00843A0610B48844203D1FFF791FB0646BF
S31508003CF002E0FFF77BFB064630462968FDF70AFE19
S31508003D000009206230462968FDF704FE0007000F07
S31508003D10606270BD0038014001464868C0B270470D
S31508003D20CAB2026070474B21C90101603021017196
S31508003D3000218171017218214181002101737047A8
S31508003D4010B51C484088030000F039FA0504111E16
S31508003D50292A2B0017488030C088FF211E31884247
S31508003D6004DA01211348418000F0E6F919E0114808
S31508003D708030C088FF210931884204DA02210D48C3
S31508003D80418000F0D9F90CE00A488030C088FD2847
S31508003D9004DA03210748418000F0CEF901E000E08B
S31508003DA000BF00BF03488030007B002801D100F027
S31508003DB0C3F910BDF002002010B53048408800282D
S31508003DC006D0012813D0022820D0032854D12CE08D
S31508003DD080210920C006FFF758F801212848FFF777
S31508003DE054F810210920C006FFF74FF844E00121D6
S31508003DF02348FFF74AF880210920C006FFF743F851
S31508003E0010210920C006FFF73EF835E08021092079
S31508003E10C006FFF73AF801211948FFF734F81021D0
S31508003E200920C006FFF72FF826E016494868CD2175
S31508003E30FDF770FDC007C00F002805D080210920B6
S31508003E40C006FFF720F80DE00E494868CD21FDF7BA
S31508003E5061FDC007C00F002804D180210920C006D3
S31508003E60FFF713F801210648FFF70DF8102109207E
S31508003E70C006FFF708F800BF00BF10BDF00200201B
S31508003E8000040048B001002010B59448007A0300E9
S31508003E9000F095F905043068AAFCFB008F48C08835
S31508003EA0FD2802DB01218D48017240218C48FEF76E
S31508003EB0E1FF00281DD08B494868FF21F531FDF741
S31508003EC029FDC007C00F002805D180210920C0069A
S31508003ED0FEF7D9FF04E080210920C006FEF7D5FFCA
S31508003EE010210920C006FEF7CEFF01217C48FEF707
S31508003EF0CAFFF0E07948C088FF211731884202DB03
S31508003F0002217648017240217548FEF7B3FF002862
S31508003F1027D074494868FF21F531FDF7FBFCC00737
S31508003F20C00F002804D101216D48FEF7ACFF03E05D
S31508003F3001216B48FEF7A9FF80210920C006FEF77C
S31508003F40A2FF10210920C006FEF79DFF63488038AE
S31508003F504088012805D0012160488038418000F05A
S31508003F60EBF8B8E05D48C088FF212531884202DDBC
S31508003F7003215A48017240215948FEF77BFF002861
S31508003F8031D058494868FF21F531FDF7C3FCC00711
S31508003F90C00F00280ED180210920C006FEF775FF44
S31508003FA001214F48FEF771FF10210920C006FEF7D0
S31508003FB06CFF0DE080210920C006FEF764FF102182
S31508003FC00920C006FEF75FFF01214548FEF75BFFA3
S31508003FD0424880384088002805D000213F4880386C
S31508003FE0418000F0A9F876E040213D48FEF742FFFF
S31508003FF000284ED0012109030920C006FEF73AFF22
S31508004000002811D180210920C006FEF73EFF0121B4
S315080040103348FEF73AFF10210920C006FEF735FFA0
S3150800402004212E48017226E02E494868FF21F53101
S31508004030FDF770FCC007C00F00280ED180210920AB
S31508004040C006FEF722FF01212548FEF71EFF1021B4
S315080040500920C006FEF719FF0DE080210920C006D9
S31508004060FEF711FF10210920C006FEF70CFF0121FB
S315080040701B48FEF708FF194880384088002808D0F2
S31508004080002116488038418001E023E002E000F074
S3150800409053F820E040211248FEF7ECFE002818D01D
S315080040A080210920C006FEF7F0FE01210C48FEF724
S315080040B0ECFE10210920C006FEF7E7FE0748803807
S315080040C04088002805D0002104488038418000F047
S315080040D033F800E000BF00BF10BD000070030020E9
S315080040E000040048B00100200348806840084000EA
S315080040F00149886070470000002C0040034880682A
S31508004100002801D0012070470020FCE7002C004061
S3150800411010B5FFF7F3FF002804D0FFF7E5FF662088
S3150800412000F002F810BD00004106490E014A116070
S3150800413070470000002C004010B57E20FFF7F4FF02
S315080041400848FEF725FD084908480180052100F0C2
S3150800415005FA06494881402202490448FEF755FDFA
S3150800416010BD000000900008FBAA0000F002002025
S315080041700FB410B503A9044B044A029800F080F85E
S3150800418010BC08BC04B01847394D0008A801002027
S315080041902021020C01D010211046020A01D0104637
S315080041A00839020901D01046091F820801D01046B5
S315080041B0891E420801D0881E7047081A704730B415
S315080041C07446641E2578641CAB4204D3635D5B00A9
S315080041D0E31830BC18471D46F8E7000010B500285C
S315080041E019DB1A4A03231B02D21883089B00D258EC
S315080041F08307DC0EFF23A3409A438B071B0E840715
S31508004200E40EA3401A43114B032424021B19840805
S31508004210A4001A5118E00E4A03071B0F083B9B0817
S315080042209B00D2588307DC0EFF23A3409A438B07D3
S315080042301B0E8407E40EA3401A43054B0407240FFC
S31508004240083CA408A4001A5110BD000000E100E0D3
S315080042501CED00E002E008C8121F08C1002AFAD1C6
S3150800426070477047002001E001C1121F002AFBD1E8
S31508004270704700000149086070470000AC01002043
S31508004280FFB58FB00F460446002606E025280AD05B
S31508004290129A11999047641C761C20780028F5D14B
S315080042A0304613B0F0BD00250121A14A009500E073
S315080042B00543641C23780846203B98401042F7D1F2
S315080042C020782E2815D1042005436078641C2A28F6
S315080042D00AD101CF641C00900BE000990A225143D1
S315080042E030394018641C0090207801463039092975
S315080042F0F3D920786C280ED004DC4C2813D06A2811
S3150800430012D104E074280ED07A280DD10BE00120D2
S315080043104005054307E00121090562780D438242FD
S3150800432001D16D18641C641C2078864669284AD019
S3150800433008DC0028B4D058286DD0632810D064282B
S3150800434008D140E070286BD0732812D0752860D049
S31508004350782860D0129A704611999047761CE5E045
S315080043603878694608720020487202A80190012030
S3150800437003E0386801900020C0433F1D69070CD54B
S31508004380002500E06D1C00998D420FDA8542F9DBA5
S315080043900199495D0029F5D108E0002500E06D1C6A
S315080043A08542FCDB0199495D0029F8D1761907E0B9
S315080043B0019801990078491C0191129A1199904720
S315080043C06D1EF5D2B2E00A20029000216802400F65
S315080043D0039102280CD001CFC117844600290DDAB3
S315080043E06246084652420021814194462D2008E043
S315080043F0FF1DFF08FF0003CF8446EFE7280504D515
S315080044002B206A46107401203CE0E8073AD02020A9
S31508004410F7E70A2000E0102000210391029007E048
S3150800442010200290002104200543082003910090E3
S315080044306802400F022810D001CF002184460020D0
S315080044400D9028071FD5704670280CD0029A1020A8
S31508004450039B42401A430CD015E0FF1DFF08FF00DE
S3150800446003CF8446EBE740206A46107401200D907E
S315080044700CE06046084306D030206A461074704641
S31508004480507402200D907046582804D029A0019037
S315080044900DA80E900DE02CA0F9E76046039B029A42
S315080044A0FDF76EFD019B84469B5C0E9A521E0E928A
S315080044B0137060460843F0D10E9805A9081A2030F3
S315080044C00190680701D5009801E001200090019944
S315080044D0884203DD01460198081A00E000200025FD
S315080044E0009006E004A8129A405D119990476D1C49
S315080044F0761C0D988542F5DB04E0129A3020119956
S315080045009047761C0099481E00900029F5DC08E0C3
S315080045100E980E990078491C0E91129A1199904797
S31508004520761C0199481E01900029F1DC641CB4E64A
S31508004530092801003031323334353637383961626B
S31508004540636465660000000030313233343536372F
S3150800455038394142434445460000000010B502463A
S315080045600023002901D1002010BD03E01488921C05
S31508004570E01883B208464C1EA1B20028F6D11846A8
S31508004580F2E70000F8B50027002600240025F748C2
S31508004590C07A012879D17E20FFF7C6FDF448C07994
S315080045A00002F349097A08430746F148467A847AAD
S315080045B00246D17A107B00F00DFD05460021EB4836
S315080045C0C172EC49781A8F4278D01EDCEA49781A0B
S315080045D08F4274D010DCE949781A8F4270D006DC15
S315080045E0442F1CD0E648381800286AD1DAE1882812
S315080045F068D08928F9D16BE1012879D0022878D0CA
S31508004600032877D00428F0D132E10300FFF7D7FD5D
S315080046100C59BDF7F559591925738B3E5B59062E6A
S3150800462009D1D848007800280AD100F0F9FF0120FE
S31508004630D449087004E0152E02D1012000F0F0FFDD
S31508004640CEE1CA4820308079002805D0C7480288BC
S315080046504188002000F03EFFC2E1002C09D1C34882
S31508004660408800231A46F0210090FE2000F067FFDC
S315080046700AE0012C08D1BD48008801230022F02158
S315080046800090FE2000F05BFFAAE1AAE1002C09D108
S31508004690BD48408800231A46F3210090FE2000F00A
S315080046A04EFF0AE0012C08D1B74880890123002271
S315080046B0F3210090FE2000F042FF91E14EE049E12F
S315080046C07EE18CE118E1002C02D1AF48458001E07B
S315080046D0AD488581AC488089FF21F531884206DAE4
S315080046E000F00CFB0022FE21F42000F05CFF77E1CD
S315080046F00CE15AE06AE0002C09D1A348808800231F
S315080047001A46F1210090FE2000F019FF0AE0012C5C
S3150800471008D19D48C08901230022F1210090FE207E
S3150800472000F00DFF5CE1002C02D19748858003E07C
S31508004730012C01D19448C58193488088FF21F53121
S3150800474088420ADC9048C089884206DC00F0D6FA1E
S315080047500022FE21F22000F026FF41E1002C09D1BB
S315080047608948C08800231A46E9210090FE2000F0F7
S31508004770E6FE09E0012C07D1192001230022E921D0
S315080047800090FE2000F0DBFE2AE1002C01D17E48D5
S31508004790C580FF202D30854206DA00F0AFFA0022E8
S315080047A0FE21EA2000F0FFFE1AE1002C0CD1764823
S315080047B000896421484380B200231A46E22100900A
S315080047C0FE2000F0BCFE00E000BF09E1002C06D187
S315080047D064212846FDF7B4F881B26B4801816A481E
S315080047E00089FF21F531884206DC00F087FA0022AD
S315080047F0FE21E32000F0D7FEF2E01EE0FFE7002CE2
S315080048000CD1614840896421484380B200231A4686
S31508004810EB210090FE2000F092FE0DE0012C0BD15A
S315080048205948008A6421484380B201230022EB21BB
S315080048300090FE2000F083FED2E0002C07D1642110
S315080048402846FDF77DF881B24F48418108E0012CE2
S3150800485006D164212846FDF773F881B24A480182D9
S3150800486000F04CFA0022FE21EC2000F09CFEB7E096
S31508004870012C14D13D48007A002807DD01213B4868
S315080048802030817100204049403948600022FE21CD
S31508004890E42000F088FE01213448017317E0002C5B
S315080048A010D1002131480173203081710022FE2188
S315080048B0E42000F078FE0020324908703249403979
S315080048C0486004E00022FE21E42000F06CFE87E048
S315080048D0002C0FD12648C07A32280CDC2448C17A2D
S315080048E02948418200F00AFA0022FE21DF2000F062
S315080048F05AFE00E000BF73E02348408A00231A46A8
S31508004900DE210090FE2000F01AFE69E0002C0FD18F
S315080049101748C07A32281CDC1548C17A1A488182A1
S3150800492000F0ECF90022FE21E12000F03CFE10E048
S31508004930012C0ED10E48C07A32280ADC0C48C17AFE
S315080049401148C18200F0DAF90022FE21E12000F0C8
S315080049502AFE45E0002C19D10B48808A00231A4606
S31508004960E0210090FE2000F0EAFD1AE07003002026
S3150800497094040020E9FE0000E0FE000056FE000058
S31508004980AB01FFFFA4010020F0010020012C08D193
S315080049901448C08A01230022E0210090FE2000F07E
S315080049A0CEFD1DE0002C07D101210F48817200229F
S315080049B002210E48FFF769F90DA0FFF7D9FB0FE0B2
S315080049C0002C0BD1FF2101310A48FCF7E6FF002035
S315080049D00849891F088002210348817200E000BF48
S315080049E000BFF8BDF0010020700300200038014028
S315080049F0313233009A040020F0B589B000200890BF
S31508004A00079006903B48C07A012871D13A488079C8
S31508004A10AA286AD13848C079322866DA3648C07971
S31508004A20002862DD3449C97908461938FDF726FA9F
S31508004A3008900898FDF774FA0446304A304BFDF79B
S31508004A403DF900222F4B01910090FDF785F803915F
S31508004A5002902D480068FDF763FA0646039B029A02
S31508004A60FDF794F905910490FDF76EFA079027492A
S31508004A700798FCF7F6FF0446FDF720FA81B22448AA
S31508004A8001830898FDF74CFA06461C4A1C4BFDF7AD
S31508004A9015F9044600221B4BFDF75EF803910290B8
S31508004AA01C480068FDF73CFA01910090039B029AA6
S31508004AB0FDF76CF905910490FDF746FA069013493F
S31508004AC00698FCF7CEFF0446FDF7F8F981B21048C0
S31508004AD0418300F013F90E48428B018B0EA0FFF7B5
S31508004AE047FB002103488172017300210148C17206
S31508004AF009B0F0BD7003002094040020091B9E5ED7
S31508004B0029CB703F0000F03F4001002000007A44A6
S31508004B10F001002044010020525F30203A20202571
S31508004B20642020525F313A2020202564200D0A0097
S31508004B3070B505460E461446002E02D0012E4AD1FF
S31508004B4020E0002D02D0012D1AD10CE060210120B1
S31508004B508007FEF70DFF002101208007FEF78CFF76
S31508004B601E4804700CE0602101208007FEF708FF4C
S31508004B70002101208007FEF788FF1948047000BF4E
S31508004B8000BF28E0002D02D0012D22D110E01348E5
S31508004B900078A0420BD0602101208007FEF7E8FECE
S31508004BA0214601208007FEF767FF0C48047010E0D5
S31508004BB00B480078A0420BD0602101208007FEF741
S31508004BC0DFFE214601208007FEF75FFF04480470D8
S31508004BD000BF00BF00BF00BF70BD00005601002027
S31508004BE05701002070B505252AE080213548FCF7D5
S31508004BF0D4FE80213348FDF7F5FE0F213148FFF733
S31508004C00ADFC3049C98B88420BD12E4800882E4905
S31508004C10884204D000F094FA00F070F800E070BD05
S31508004C200EE02AA0FFF7A4FA002407E06100254851
S31508004C30425A214628A0FFF79BFA641C802CF5DB14
S31508004C402846691ECDB20028CFD100BF05252CE025
S31508004C5080211C48FCF7A1FE80211A48FDF7E0FEDA
S31508004C600F211848FFF77AFC1649C98B88420DD1DF
S31508004C70144800881449884204D000F061FA00F00C
S31508004C803DF802E000F03AF8C9E70EE015A0FFF794
S31508004C906FFA002407E061000A48425A214614A028
S31508004CA0FFF766FA641C802CF5DB2846691ECDB230
S31508004CB00028CDD100BF00F043FA00F01FF800BF6E
S31508004CC0ADE70000F0010020FBAA00004641554C64
S31508004CD054215F31000000002564202025640D0A58
S31508004CE0200000004641554C54215F320000000068
S31508004CF05F322564202025640D0A200010B57E2029
S31508004D00FFF712FAFDF72EFF09490A4801800F211D
S31508004D10FFF724FC0749C88380210648FDF7BCFE37
S31508004D207E20FFF701FA80210248FDF7C1FE10BD7B
S31508004D30FBAA0000F001002070B504460D46E1B25A
S31508004D400548FEF7EDFF00BF01210348FEF78BFF7C
S31508004D500028F9D0204670BD0038014070B50446D9
S31508004D60002599480088FA280ADD00209649088017
S31508004D7096490870FF2101319348801DFCF70DFE06
S31508004D80924800780300FFF71AFA08052031425BBB
S31508004D90D5EFEDEC7E2C11D100208B49088001203F
S31508004DA08A490870884801880088401C864A10800D
S31508004DB0901D445400201146C87002E00020824924
S31508004DC00880002080490871FBE07F480188008838
S31508004DD0401C7D4A1080901D445402207B4908706F
S31508004DE010460079001911460871EAE076480188EC
S31508004DF00088401C744A1080901D4454032073494F
S31508004E00087010460079001911460871D9E06E48F5
S31508004E1001880088401C6C4A1080901D4454042068
S31508004E206A49087010460079001911460871084643
S31508004E30C470C078002802D1052064490870C0E013
S31508004E4061484079012856D15E2C1CD15E4800790C
S31508004E507E305D4908717E215B4802880088401CC7
S31508004E60594B1880981D8154801FC078401EC0B2C7
S31508004E701946C870002802DC05205449087000202D
S31508004E805149487155E05D2C1CD14F4800797D3059
S31508004E904D4908717D214C4802880088401C4A4BC0
S31508004EA01880981D8154801FC078401EC0B21946CC
S31508004EB0C870002802DC05204449087000204249D1
S31508004EC0487136E04048007900193F49087108469C
S31508004ED001880088401C3C4A1080901D4454801F5D
S31508004EE0C078401EC0B21146C870002821DC0520D3
S31508004EF0364908701DE07D2C03D1012032494871DE
S31508004F0017E03148007900192F49087108460188C9
S31508004F100088401C2C4A1080901D4454801FC0787D
S31508004F20401EC0B21146C870002802DC0520274979
S31508004F30087046E024480079C043401CC5B2A54223
S31508004F4003D106202149087002E007201F4908708E
S31508004F501D4801880088401C1B4A1080901D445437
S31508004F602FE02DE01DE0FFE7174801880088401C68
S31508004F70154A1080901D44547E2C08D101211448EE
S31508004F80C1720020114608801049087008E0002008
S31508004F900D49088000210E48C17200200B4908708F
S31508004FA00FE0002009490870074801880088401C5E
S31508004FB0054A1080901D445400201146088000E0E0
S31508004FC000BF00BF70BD000094040020A3010020AC
S31508004FD07003002070B50246002013460C461D02D9
S31508004FE0FF26360235402543284670BD86B004465E
S31508004FF00D4626686768A0680590E06804902069F1
S31508005000039060690290A0690190E069009017A07A
S31508005010FFF7AEF831461BA0FFF7AAF839461CA0E1
S31508005020FFF7A6F81DA00599FFF7A2F81EA0049998
S31508005030FFF79EF81FA00399FFF79AF820A0029998
S31508005040FFF796F823A00199FFF792F826A0009992
S31508005050FFF78EF82948416A29A0FFF789F82946FB
S315080050602BA0FFF785F800BFFEE700005B486172DA
S3150800507064206661756C742068616E646C65725D27
S315080050800D0A00005230203D2025780D0A00000048
S315080050905231203D2025780D0A0000005232203D6D
S315080050A02025780D0A0000005233203D2025780D72
S315080050B00A000000523132203D2025780D0A0000F2
S315080050C0537461636B6564204C52203D2025780D2E
S315080050D00A000000537461636B6564205043203DE9
S315080050E02025780D0A000000537461636B656420FF
S315080050F0505352203D2025780D0A000000ED00E0AF
S315080051005343425F53484353523D25780D0A0000E6
S3150800511043757272656E74204C52203D2025780DB9
S315080051200A000000044905480180002141805F21EA
S315080051308180C18001817047FBAA0000F00200202F
S3150800514000B5124912480180FF2141800F210181D3
S31508005150A021C180D22181801E214181AF21C18138
S315080051608C210182BE2181810A49018309492331A3
S315080051704183052141820A218182C18200218183DE
S315080051800F21FFF7EBF90249C88300BDFBAA00000F
S31508005190F00100205A25000010B55548C07B0128AB
S315080051A026D154494868C821FCF7B4FBC007C00F8C
S315080051B0002805D180210920C006FDF764FE0DE010
S315080051C04C494868C821FCF7A5FBC007C00F002852
S315080051D004D080210920C006FDF757FE10210920BA
S315080051E0C006FDF750FE01214348FDF74CFE10BDF1
S315080051F03F48007B012878D13D4820308079002837
S3150800520002D0012834D10BE040213B48FDF732FE9D
S31508005210002802D1FEF7D0FD01E0FEF735FE63E077
S3150800522034494868FF21F531FCF774FBC007C00F05
S3150800523000280ED180210920C006FDF726FE01218F
S315080052402D48FDF722FE10210920C006FDF71DFE98
S315080052500DE080210920C006FDF715FE1021092062
S31508005260C006FDF710FE01212348FDF70CFE3BE0C2
S315080052701F4820308079052827D11E494868FF2114
S31508005280F531FCF747FBC007C00F00280ED1802177
S315080052900920C006FDF7F9FD01211748FDF7F5FDC0
S315080052A010210920C006FDF7F0FD1CE08021092029
S315080052B0C006FDF7E8FD10210920C006FDF7E3FD4D
S315080052C001210D48FDF7DFFD0DE080210920C0060C
S315080052D0FDF7DBFD01210848FDF7D7FD1021092060
S315080052E0C006FDF7D2FD00BF00BF00BF7FE7000084
S315080052F070030020B001002000040048FEF762FA9F
S3150800530000F0C2F8FDF7C6FFFEF756FDFDF7C2FA34
S31508005310FDF760F80B20FCF79BFF0920FCF798FFC8
S315080053200320FCF795FF01215248FDF7F9F84B20B9
S315080053300002FDF719FAFDF727FFFEF779FA0D21A6
S315080053406320FEF7A3FA01214B4801730021C173BC
S31508005350FFF748FCFEF7E6FB8AE04748807A002814
S315080053600AD1FDF705F9FFF717FFFFF70BF9FDF768
S315080053703FFF00F093FD78E03F48807A012836D158
S31508005380002301221946184600F0AAF900231A46F6
S315080053901946184600F0A4F9384840683849884242
S315080053A004D908213748FDF76EFD1DE033494868E2
S315080053B0FF21F531FCF7AEFAC007C00F00280ED161
S315080053C080210920C006FDF75EFD10210920C006D0
S315080053D0FDF759FD01212B48FDF755FD04E0102185
S315080053E00920C006FDF751FDFDF76AF93DE02248A0
S315080053F0807A022839D1FDF7BBF8FDF7F9FE0023BC
S3150800540001221946184600F06BF900231A46194678
S31508005410184600F065F9194840681949884204D9C0
S3150800542008211848FDF72FFD1DE014494868FF219B
S31508005430F531FCF76FFAC007C00F00280ED180219E
S315080054400920C006FDF71FFD10210920C006FDF73B
S315080054501AFD01210B48FDF716FD04E0102109206D
S31508005460C006FDF712FDFFF7C7FA7E20FEF75CFEC1
S3150800547073E700000024014070030020B0010020FB
S31508005480204E00000004004810B540210E48FCF7E5
S3150800549084FA40210C48FDF7E1FA05210A48FFF78E
S315080054A05DF809494989884209D1084800880849A8
S315080054B0884208D0FFF736FEFEF73EFE03E0FFF708
S315080054C031FEFEF739FE10BDF0020020F001002083
S315080054D0FBAA0000F7B5A0B00C4615468021684621
S315080054E0FCF75BFA002700267E2168460170FE213C
S315080054F04170EF2181700721C17020990171002147
S31508005500417184712112C1710121017245722912FA
S315080055108172012605E06846805DC019C7B2701C15
S31508005520C6B20B2EF7DBF843401CC1B26846C172FF
S315080055307E2101730D21FEF761FB23B0F0BDFFB597
S3150800554085B005460E460E9F0020019002900390F6
S315080055500490009000247E21684601714571867189
S315080055600421C1710799017208994172877239122B
S31508005570C172012407E001A8015D00980818C0B2AD
S315080055800090601CC4B2082CF5DB0098C043401C90
S31508005590C1B2684601737E2141730A2101A8FEF74C
S315080055A02DFB09B0F0BDF7B584B005460E460020C0
S315080055B00090019002900390002700247E216846FF
S315080055C00170467085700121C17069460698087198
S315080055D0012405E06846005DC019C7B2601CC4B264
S315080055E0052CF7DBF843401CC1B2684641717E21A1
S315080055F081710721FEF702FB07B0F0BD70B50446BE
S315080056000D467E20FEF790FD03E02078641CFEF729
S31508005610E5FA2846691E8DB20028F6D170BD00004D
S3150800562030B5A1B00446802101A8FCF7B6F90025DB
S31508005630002C02D0012C20D10FE07E216846017192
S3150800564000214171442181711321C171152210492C
S3150800565002A8FCF789F9192510E07E216846017130
S31508005660FE214171442181713321C17136220949D4
S3150800567002A8FCF779F93A2500E000BF00BF802DA3
S3150800568003DA294601A8FFF7B9FF21B030BD0000AB
S31508005690580100206D010020F8B506460C46FCF7B7
S315080056A073FD051E0F4600D00120014349000B4833
S315080056B04908411AC90F0DD0002E01D0012100E07A
S315080056C000210C4361004908401AC00F02D101208D
S315080056D0FEF7D0FD28463946F8BD00000000F07FE9
S315080056E0FFB58DB005460E4600200B9000240A90A3
S315080056F009900890FE480078642803D0FD48007891
S31508005700642803D10121FC48017402E00021FA480B
S3150800571001740F98002802D0012871D197E0F74844
S31508005720C089B04202D1F548C48A00E00524052C98
S3150800573001DC052402E0322C00DB0524301BA842DC
S315080057400DDDED48407D00284CD1EC4840384068D6
S31508005750EA49403988610121E748417542E0301934
S31508005760A8423FDCE448407D01283BD1E24820308E
S31508005770007901282FD1E14840384068DF4940398F
S315080057808969401ADE4988420DD2DB48803800898B
S31508005790462820DDD84880380089801E81B2D64840
S315080057A08038018117E0D54840384068D3494039E8
S315080057B08969401A7D21890188420CD9CE488038EA
S315080057C000895F2807DACC4880380089801C81B2B6
S315080057D0C948803801810121C7482030017100215C
S315080057E020384175C448407D012826D1C048007834
S315080057F0C0490978884204DA0020BD4908701FE0CC
S3150800580038E3301BA84203DD6420B949087017E065
S315080058101E2C03DD6420B649087011E0B648203016
S315080058200079002803D16420B149087008E0B2481D
S315080058308038007AAE49087002E00020AC4908704A
S31508005840AB48027810990F98FFF772F912E3AA4845
S3150800585020308079012858D1A8484088B04202D122
S31508005860A648448A00E00A24A4484188408A081ABF
S31508005870A84209DBA14840384068A04940398862F7
S315080058800020A049087017E09C484088A84213DC0D
S315080058909C48007800280FD19748C188C183012009
S315080058A09849087095484038406894494039896A4B
S315080058B0401A92494039086290488188808A081AB5
S315080058C0A84209DB0020904908708C484038406897
S315080058D08A494039C8623CE088488088A84238DC52
S315080058E089480078002834D18348C188018401207A
S315080058F08549087081484038406880494039C96AF6
S31508005900401A7E494039486223E07B482030807936
S31508005910022808D179484088B04202D17748448A9B
S3150800592017E00A2415E0744820308079032808D146
S3150800593072488088B04202D17048848A09E00A24F5
S3150800594007E06E488088B04202D16C48848A00E03D
S315080059500A24052C01DC052402E0322C00DB322463
S31508005960301BA84218DB654840384068634940390F
S31508005970C8610020086348635F488580807D0028E9
S3150800598006D11E215C48203081700121203881759E
S3150800599000215948C17424E13019A8427EDC5648D2
S315080059A0807D0128F7D1544820308079012876D1A6
S315080059B05148203040790028F9D15048408A0A28B1
S315080059C00BDB4E494039086AFCF763FA07464F492C
S315080059D0FCF784F84E4908601EE04848408A0A28C1
S315080059E00FDA4648408A07280BDD44494039086AD9
S315080059F0FCF74FFA07464749FCF770F84449086030
S31508005A000AE03E494039086AFCF743FA0746424924
S31508005A10FCF764F83E4908603749C88BFCF739FA41
S31508005A2035490790C88BFCF734FA05903848016861
S31508005A300598FCF716F806900799FCF712F807463A
S31508005A40FCF76EFA354A03C22B49C88BFCF728FACD
S31508005A5003910290314903C9FFF71EFE0191009098
S31508005A60039B029AFCF792F900222D4B05910490AC
S31508005A70FCF724F907910690FCF734FA81B21E4820
S31508005A80803881801D494039486AFCF702FA074682
S31508005A902049FCF723F81E49086001E0A0E053E01E
S31508005AA01549088CFCF7F5F913490790088CFCF79B
S31508005AB0F0F90590164801680598FBF7D2FF06909D
S31508005AC00799FBF7CEFF0746FCF72AFA134A03C2E3
S31508005AD00949088CFCF7E4F9039102900F4903C9B8
S31508005AE0FFF7DAFD01910090039B029A1AE0000085
S31508005AF0D9000020DA00002070030020F001002001
S31508005B0070170000CC000020CD00002000803B4527
S31508005B10C40000200000FA440080BB44D0000020E6
S31508005B2000005940FCF732F90022D44B0591049045
S31508005B30FCF7C4F807910690FCF7D4F981B2D0486F
S31508005B40C1800121A0304171CE484068CD49C9695C
S31508005B50401ACD4988421FDDC948A03080790228FD
S31508005B600AD1C74880885F2831DAC5488088801CF2
S31508005B7081B2C34881802AE0C148A03080790328D1
S31508005B8025D1BF48C0885F2821DABD48C088801C57
S31508005B9081B2BB48C1801AE0BA484068B949C969A8
S31508005BA0401A7D214901884211DAB6484068B5494C
S31508005BB0C969401A00280ADDB148A0308079022850
S31508005BC005D0AF48A0308079032800D000BF002157
S31508005BD0AB4880308175AB484068AA49C86100E087
S31508005BE000BFA7488030807D01287DD1A448A03019
S31508005BF08078A6490978884204DA0021A048A030AE
S31508005C00817022E1301BA84207DD64219C48A03040
S31508005C10C17001212038017417E19948A0308079B4
S31508005C20012804D0022815D003287DD188E0301930
S31508005C30401BA04209DA3019401B201A5F21081AB6
S31508005C40C1B28F48A030C17003E05F218C48A030F4
S31508005C50C170CEE08B49086B7D21C900FBF75AFE5F
S31508005C602746E10FC919491048438019001B80B21D
S31508005C7008908448006B8349496B401A7D21C90006
S31508005C80884235D97F48006B7E4948637C48803016
S31508005C908088A84206DD7A4880880A3081B278482A
S31508005CA0818020E07649803189886A1AE10F0919CE
S31508005CB04910491C8A4206DA71488088801C81B2DC
S31508005CC06F4881800FE06E49803189886A1AE10F32
S31508005CD009194910891C8A4205DD69488088801E91
S31508005CE081B26748818000E084E06548803085801D
S31508005CF06448006B6649884209D9002061490863EF
S31508005D0048635F488088401D81B25D4881805C4851
S31508005D100179A030C1705B4840685A49C969401A80
S31508005D205B4988420BDD00E05EE055488088401DEF
S31508005D3081B253488180534840685249C86158E047
S31508005D405048006B4F49496B401A7D21C90088426B
S31508005D5033D94C48006B4B494863494880308088A2
S31508005D60A84206DD4648C0880A3081B24448C18048
S31508005D7020E04349803189886A1AE10F09194910D8
S31508005D80491C8A4206DA3E48C088801C81B23C48D3
S31508005D90C1800FE03A49803189886A1AE10F0919EA
S31508005DA04910891C8A4205DD3548C088801E81B2A3
S31508005DB03348C18032488030858031488179A030A7
S31508005DC0C170304840682F49C969401A314988422C
S31508005DD009DD2B48C088401D81B22948C180294861
S31508005DE040682849C86104E032212548A030C170BE
S31508005DF000BF2AE02248A0308079012821D1301935
S31508005E00A84219DB1E480179A030C1703019801EDE
S31508005E10A8420DDD20480078002816D11848808849
S31508005E20401D81B21648818001201B4908700CE08C
S31508005E3000201949087008E000211148A030C170F7
S31508005E4003E00A210E48A030C1700D48A0308079C1
S31508005E50012807D10A48A030C27810990F98FEF792
S31508005E6067FE06E00648A030827810990F98FEF77C
S31508005E705FFE00BF00BF0B9811B0F0BD000059408F
S31508005E80F0020020B001002070170000D9000020A1
S31508005E9088130000581B0000D800002010B5FE48E3
S31508005EA08079002858D0FC4820384088FF217D3169
S31508005EB0884204DCF8482038008888420ADDF6481B
S31508005EC02038C07B002805D1F44948600121F248F2
S31508005ED02038C173F148806BF14988420AD9EE48E7
S31508005EE02038C07B002805D1EC4948600121EA48E2
S31508005EF02038C173E8482038C07B01282CD1E648F1
S31508005F002038007B012827D100230122194618468C
S31508005F10FFF7E6FB00231A4619461846FFF7E0FB8B
S31508005F20DE4840687D210901884214D90020DB49F2
S31508005F30486010210920C006FCF7A5FF802109202A
S31508005F40C006FCF7A0FF0121D648FCF79CFF0021FC
S31508005F50D1482038017310BDCF482038007B00286F
S31508005F6059D110210920C006FCF78DFF8021092090
S31508005F70C006FCF788FF0121CA48FCF784FF002108
S31508005F80C54881710023012219461846FFF7A8FB68
S31508005F9000231A4619461846FFF7A2FBBF48406871
S31508005FA0FF21F531884204D22021BE48FCF76DFF57
S31508005FB020E22021BB48FCF766FFB8484068BA498A
S31508005FC08842F5D9B4482038007D002812D1B34854
S31508005FD040687D214901884201D2FDF7B1FE0821BA
S31508005FE0B048FCF750FF0021AB482038C173203079
S31508005FF001710BE04021AB48FCF73CFF002805D0B7
S315080060000021A54881710121203801737D204001B6
S31508006010A2494860EEE1A04880790300FEF7CFF870
S3150800602006044FA6E7FDFC4E00219B48417100235C
S31508006030012219461846FFF753FB00231A4619464C
S315080060401846FFF74DFB94482038807A012809D175
S31508006050924800699549884203D900218E4820381C
S31508006060817278E78D4840687D210901884221D9E7
S3150800607000208A49486040218A48FCF7FBFE002830
S3150800608009D1FDF75DFE08218648FCF7FCFEFF20D6
S31508006090F530FCF7C1FB10210920C006FCF7F3FE1A
S315080060A080210920C006FCF7EEFE01217D48FCF799
S315080060B0EAFE03E008217B48FCF7E7FE99E177480A
S315080060C04068FF21F531884204D220217548FCF743
S315080060D0DCFE03E020217348FCF7D5FE6F494868CB
S315080060E07D21C900FBF716FC23281FD26B49486897
S315080060F07D21C900FBF70EFC192817D966482038F8
S315080061000188FF3881384088814207DA624820389A
S315080061104188FF3881384088814216DB00205F4974
S315080061204860C86102215C4881710EE05B49486895
S315080061307D21C900FBF7EEFB232806D3002057492B
S315080061404860C861022154488171544A40325188D6
S31508006150FF328132508801231A46FFF7C1FA00231D
S315080061601A4619461846FFF7BBFA42E14B484068FB
S31508006170FF21F531884204D220214A48FCF785FEE2
S3150800618003E020214748FCF77EFE4448416840303A
S3150800619000897D22D2005043814210D23F4A4032C4
S315080061A05188FF328132508801231A46FFF798FA40
S315080061B000231A4619461846FFF792FA0DE0002101
S315080061C03548203881750020344948600121324815
S315080061D02038C17403212030817130480088FF219E
S315080061E0F531884202DD00202C49088001E12A4861
S315080061F020384088FF217D31884204DC2648203833
S31508006200008888420FDD0023012219461846FFF749
S3150800621067FA00231A4601E07BE02BE01946184688
S31508006220FFF75EFA25E01D4948687D21C900FBF79E
S3150800623071FB1A4940314989884210D2174A4032BF
S315080062409188FF328132508801231A46FFF748FAAF
S3150800625000231A4619461846FFF742FA09E00020B5
S315080062600E49486000210C482038817504212030E9
S315080062708171BEE0084820384088FF217D31884278
S3150800628004DC05482038008888421ADD00230122EC
S31508006290194618460CE0000090030020B0010020C3
S315080062A07011010000040048B80B000088130000B4
S315080062B0FFF716FA00231A4619461846FFF710FA8A
S315080062C026E04D4948687D21C900FBF723FB4A496A
S315080062D04031098A0F39884214D2474A4032D18957
S315080062E0FF328132108801230022FFF7F9F9424A6A
S315080062F04032D188FF328132508801231A46FFF78F
S31508006300EFF905E000203C49486005213B488171CA
S315080063106FE039484068FF21F531884204D22021D0
S315080063203748FCF7B2FD0FE033484068FF21F531E6
S31508006330884209D9304840684B21C900884203D2AF
S3150800634020212F48FCF79FFD2B4840682D4988429D
S315080063502DD22A4820384088FF211931884204DC8A
S3150800636026482038008888420CDD00230122194679
S315080063701846FFF7B5F900231A4619461846FFF7D7
S31508006380AFF935E01C4A4032D189FF328132108894
S3150800639001230022FFF7A4F9174A4032D188FF32B9
S315080063A08132508801231A46FFF79AF920E0202106
S315080063B01348FCF76AFD104840681349884217D30A
S315080063C000200D49486000210C488171203801736E
S315080063D00023012219461846FFF782F900231A46B8
S315080063E019461846FFF77CF920210548FCF74BFDAE
S315080063F000BF00BF00BFAEE5B0010020900300203B
S3150800640000040048A4380000983A00002C640008EC
S31508006410C0000020F0000000544200081C65000877
S31508006420B0010020F00700006442000800000000E8
S31508006430000000000000000000000000000000004E
S31508006440000000000000000000000000000001023B
S3150800645003040102030406070809000000A24A040F
S3150800646000000000000000000102030406070809F6
S31508006470000000000000000000000000000000000E
S3150800648004000000010000000000000000000000F9
S3150800649000000000000000000000000000000000EE
S315080064A000000000000000000000000000000000DE
S315080064B000000000000000000000000000000000CE
S315080064C00000000000011058594C4C303131327828
S315080064D078787878787878CB7E00011058594C4CC3
S315080064E030313132787878787878787804013205DE
S315080064F0054C4C303131061459413230303532387A
S315080065004834353034324178787878787D5D7E0045
S3110800651000000000000000000000000071
S705080018C515
